:100000000C94EA030C9409040C9409040C9409045C
:100010000C9409040C9409040C9409040C9409042C
:100020000C9409040C9409040C9409040C9409041C
:100030000C9409040C9409040C9409040C9409040C
:100040000C9409040C940B040C9409040C940904FA
:100050000C9409040C9409040C9409040C940904EC
:100060000C9409040C944E0D0C941A0D0C94090474
:100070000C9409040C94C3070C9409040C9409040F
:100080000C9409040C9409040C9409040C940904BC
:100090000C9409040C9409040C9409040C943A0F70
:1000A0000C9409040C9409040C9409040C9409049C
:1000B0000C9409040C9409040C9409040C9409048C
:1000C0000C9409040C9409040C9409040A003039B6
:1000D0003A33363A313000202F20004F637420200D
:1000E000312032303130000A6F6E2000323030392A
:1000F00030333039002072656C656173653A2000D9
:10010000312E362E360020616E64204156522D4C21
:100110004942433A2000342E332E32004275696C36
:10012000742077697468204156522D4743433A2022
:10013000000A0A3831303020446562756720536305
:10014000686E6974747374656C6C650A00010000F4
:1001500001091100E4010800A89C6FDE5374727558
:10016000636B20496E6E6F76617469766520537992
:100170007374656D6520476D6248C75349533831C4
:100180003030C3303031C4383130300000C100006D
:1001900000000000FE010800DE53747275636B20DE
:1001A000496E6E6F766174697665205379737465F4
:1001B0006D6520476D6248C753495338313030C4AC
:1001C00038313030C476312E30C330303100000049
:1001D00000C10000E8C002065ADE5A3100160005D0
:1001E000C00215AD7C5A31001900008001E4FFFF08
:1001F00000210000FD00211000FDC0821ABFE55A59
:1002000031002D00FF01050000010002F000E1F5C2
:100210000500E1F50500E1F50500005112120000AE
:10022000002B000000C10000C75349533831303063
:100230000100510132000000C1000340F26F0700CD
:1002400000000700000000000000000000000000A7
:10025000000000000000000000000000000000C7D7
:10026000486F7453776170000000000000000000C8
:100270000200510130000001C10003540101FF7F61
:1002800000703F0080010000010600040C0000190E
:1002900046007DC9555046D8DDE70505000000C57C
:1002A00074465047410000000000000000000000BC
:1002B0000300510131000002C10003540101FF7F1E
:1002C00000703F0080010000010600040C000019CE
:1002D00046007DC9555046D8DDE70505000000C63B
:1002E00074506F776572000000000000000000008D
:1002F0000400510130000003C10003540201FF7FDC
:1003000000703F0000040000360200040CD0077F9C
:10031000EFABFF00F7F2E9A2A7AB0202000000C5B5
:10032000752B313256000000000000000000000074
:100330000500510131000004C10003540201FF7F98
:1003400000703F0000040000A10200040CC0077F01
:10035000EFABFF00F7F2E9A2A7AB0202000000C674
:10036000752B332E33560000000000000000000003
:100370000600510131000005C10003540201FF7F56
:1003800000703F0000040000620200040CC0077F00
:10039000EFABFF00F7F2E9A2A7AB0202000000C634
:1003A000752B312E385600000000000000000000C0
:1003B0000700510131000006C10003540201FF7F14
:1003C00000703F0000040000620200040CC0077FC0
:1003D000EFABFF00F7F2E9A2A7AB0202000000C6F4
:1003E00075436F6D626F00000000000000000000A8
:1003F000708A728E9290748C76989C9AA0A4889E33
:10040000868478947A9682807C7EA270726F633A3A
:1004100020756E6B6E6F776E0A0070726F633A2094
:100420004E4554464E5F5049434D473A20434D4454
:100430005F4745545F434C4F434B5F5354415445D2
:100440000A0070726F633A204E4554464E5F504921
:10045000434D473A20434D445F4745545F414D4328
:100460005F504F52545F53544154450A0070726FAD
:10047000633A204E4554464E5F5049434D473A201B
:10048000434D445F5345545F414D435F504F525479
:100490005F53544154450A0070726F633A204E45D1
:1004A00054464E5F5049434D473A20434D445F46C2
:1004B00052555F434F4E54524F4C5F43415041425F
:1004C0000A0070726F633A204E4554464E5F5049A1
:1004D000434D473A20434D445F4745545F4445569A
:1004E0005F4C4F43414C5F5245435F49440A0070A3
:1004F000726F633A204E4554464E5F5049434D4714
:100500003A20434D445F4745545F4652555F4C4542
:10051000445F53544154450A0070726F633A204E51
:100520004554464E5F5049434D473A20434D445F42
:100530005345545F4652555F4C45445F53544154B4
:10054000450A0070726F633A204E4554464E5F5024
:1005500049434D473A20434D445F4745545F4C451E
:10056000445F434F4C4F525F43415041420A007039
:10057000726F633A204E4554464E5F5049434D4793
:100580003A20434D445F4745545F4652555F4C45C2
:10059000445F50524F50530A0070726F633A204EBE
:1005A0004554464E5F5049434D473A20434D445FC2
:1005B0004652555F434F4E54524F4C0A0070726F73
:1005C000633A204E4554464E5F5049434D473A20CA
:1005D000434D445F4745545F5049434D475F505238
:1005E0004F50530A0070726F633A204E4554464E86
:1005F0005F53544F524147453A20434D445F575251
:100600004954455F4652555F444154410A00707257
:100610006F633A204E4554464E5F53544F52414704
:10062000453A20434D445F524541445F4652555F31
:10063000444154410A0070726F633A204E4554465B
:100640004E5F53544F524147453A20434D445F4714
:1006500045545F4652555F494E565F415245415F92
:10066000494E464F0A0070726F633A204E45544619
:100670004E5F53454E535F4556454E543A20434DC9
:10068000445F4745545F53454E534F525F52454177
:1006900044494E470A0070726F633A204E455446F3
:1006A0004E5F53454E535F4556454E543A20434D99
:1006B000445F5245535F4445564943455F53445256
:1006C0005F5245500A0070726F633A204E4554469F
:1006D0004E5F53454E535F4556454E543A20434D69
:1006E000445F4745545F4445564943455F53445230
:1006F0000A0070726F633A204E4554464E5F534570
:100700004E535F4556454E543A20434D445F47454E
:10071000545F4445564943455F5344525F494E46F2
:100720004F0A0070726F633A204E4554464E5F5335
:10073000454E535F4556454E543A20434D445F5015
:100740004C4154464F524D5F4556454E540A007039
:10075000726F633A204E4554464E5F53454E535F89
:100760004556454E543A20434D445F4745545F45F6
:1007700056454E545F52454345495645520A00700E
:10078000726F633A204E4554464E5F53454E535F59
:100790004556454E543A20434D445F5345545F45BA
:1007A00056454E545F52454345495645520A0070DE
:1007B000726F633A204E4554464E5F4150503A2086
:1007C000434D445F4745545F4445564943455F495F
:1007D000440A000011241FBECFEFD1E2DEBFCDBF1F
:1007E00012E0A0E0B2E0E8EBF5E200E00BBF02C0EF
:1007F00007900D92AC33B107D9F715E0ACE3B2E046
:1008000001C01D92AB3AB107E1F70E948A040C9433
:10081000DA120C9400001F920F920FB60F9211245F
:100820002F938F939F9380917F0329B12095282741
:1008300090913D029223909590933D0280913C02CD
:100840008223892780933C029223982380917F03FF
:10085000892780937F032091380380917F03892328
:10086000822B809338032091360380917F038095FB
:100870009823922B9093360380913F0290914002EF
:1008800001969093400280933F02885E934091F4DA
:1008900091E090934C021092400210923F0280919E
:1008A0003E028F5F80933E02853021F490933703A0
:1008B00010923E02809141028F5F809341028A3004
:1008C00029F481E080933903109241029F918F9126
:1008D0002F910F900FBE0F901F901895F894909144
:1008E000380389239091380398279093380378949C
:1008F0000895F894909136038923909136039827B0
:100900009093360378940895F89490917F037894A7
:10091000892308952F923F924F925F926F927F9218
:100920008F929F92AF92BF92CF92DF92EF92FF92FF
:100930000F931F93CF93DF930E94CB0C0E94B407B9
:100940000E94D30F8DE692E090933C0380933B038B
:100950008DE393E09093E9028093E8028CEE92E0BD
:10096000909364028093630289E0809381008FE317
:100970009FE1909389008093880082E080936F00CC
:1009800013980B9A2D9885B1806C85B984B1806ECF
:1009900084B988B18A7F88B987B1856087B980E2D8
:1009A000809356028DE492E06DEC72E048ED52E0E7
:1009B0000E9488108DE492E060E041E050E00E94E7
:1009C000941080E48093B8028FEA92E065E672E0CA
:1009D0004EE253E00E9488108FEA92E060E041E02E
:1009E00050E00E94941080E88093890380E893E0AF
:1009F00065EC72E040EE52E00E94881080E893E0DF
:100A000060E043E050E00E94941080E893E060E0F2
:100A100040E050E00E9494101092EA027894109204
:100A20003A031092D70281E391E00E94BE0D8CE15F
:100A300091E00E94BE0D86E191E00E94BE0D86E02D
:100A400091E00E94BE0D80E091E00E94BE0D85EF16
:100A500090E00E94BE0D8CEE90E00E94BE0D87EEED
:100A600090E00E94BE0D8BED90E00E94BE0D87EDE0
:100A700090E00E94BE0D8EEC90E00E94BE0D8CECCA
:100A800090E00E94BE0D0E9430088093EB020E940D
:100A90002A0F80E092E00E94760D8091EB020E9486
:100AA000C50E81E192E00E94760D80E28093A00362
:100AB0001092A1032EE088E190E00FB6F894A8957B
:100AC000809360000FBE2093600000E01FEFC0E045
:100AD000D0E0FF24F394F0E13F2EE2E0EE2E74E04C
:100AE000D72E62EFC62E5FE6552E4BE0442E3CEE2D
:100AF000A32E32E0B32E2DE3622E23E0722E98EC6B
:100B0000892E912C83E0282EA895E0913B03F0914B
:100B10003C03808187FD11C0E091E802F091E90279
:100B2000808187FD0AC0E0916302F09164028081B8
:100B300087FD03C010924B0202C0F0924B02F89462
:100B400090913803947080913803892780933803FB
:100B50007894992369F4F894909136039470809175
:100B600036038927809336037894992309F44BC080
:100B700080913A03882309F046C0E0916302F09126
:100B800064028091A0038283E0916302F091640289
:100B90003382E0916302F09164028091EB028583DD
:100BA000E0916302F09164020683E0916302F091A8
:100BB0006402E782E0916302F0916402D086E091E2
:100BC0006302F0916402C186E0916302F0916402D5
:100BD0001286E0916302F09164025386F89480914A
:100BE0007F037894E0916302F091640282FF02C077
:100BF000148601C0F4860C5FE0916302F0916402F8
:100C00004182F0923A038091D702882309F445C0CB
:100C100080913A03882309F040C0E0916302F0918B
:100C200064028091A0038283E0916302F0916402E8
:100C30003382E0916302F09164028091EB0285833C
:100C4000E0916302F091640206830C5FE09163021D
:100C5000F0916402E782E0916302F0916402D08631
:100C6000E0916302F0916402C186E0916302F09129
:100C700064021286E0916302F09164025386E0916F
:100C80006302F0916402E486E0916302F0916402F1
:100C90004182F0923A031092D70280914C0288234D
:100CA00061F080E969E472E00E945C1082E965ED20
:100CB00072E00E945C1010924C0280914B028823DB
:100CC00069F580913A03882349F1B092E902A09234
:100CD000E802C5010E948C088091E8029091E90227
:100CE0000E94B5088823A1F088E592E004C0F401D1
:100CF0003197F1F701970097D1F78091E802909131
:100D0000E9020E94B508882319F088E592E0EFCF48
:100D10007092E9026092E80210923A03E0913B037C
:100D2000F0913C03808180FF44C0CF010E94D6082F
:100D3000E0913B03F0913C0390819E7F9083882358
:100D4000C1F580913B0390913C030E948608882363
:100D500071F56091E8027091E90280913B039091F6
:100D60003C030E940709882321F18091E8029091B9
:100D7000E9020E948C088091E8029091E9020E94A9
:100D8000B5088823B1F088E592E004C0F4013197FA
:100D9000F1F701970097D1F78091E8029091E9026D
:100DA0000E94B508882329F088E592E0EFCF1092E1
:100DB0003A0380913703882311F010923703809112
:100DC0003903882309F4A0CE8DE492E00E94191122
:100DD0008FEA92E00E94191180E893E00E941911B5
:100DE0008091EA02833049F1843028F4813071F037
:100DF0008230E0F409C0853079F1853038F18630F1
:100E000069F18730B9F52CC0139834C013988091DC
:100E10009603909197038C5B924060F12196C83CB9
:100E2000D10541F5E092EA02139A24C0009922C04C
:100E3000019B20C02092EA021BC02196C536D10535
:100E4000C8F03A983898D092EA0214C0339B12C086
:100E500085E08093EA020EC000000CC0389A0AC0F8
:100E600087B1856087B91398F092D7021092EA0291
:100E7000C0E0D0E08091EA02181709F472C0823015
:100E800089F1833028F4882369F0813049F41AC04D
:100E9000853009F447C0873009F454C0843091F19B
:100EA000182F5FC08FEA92E060E041E050E00E94BE
:100EB000941080E893E060E040E050E00E949410DD
:100EC00010E04FC08FEA92E060E041E050E00E9405
:100ED000941080E893E060E040E050E00E949410BD
:100EE00011E03FC08FEA92E060E042E050E00E94F3
:100EF000941080E893E060E040E050E00E9494109D
:100F000012E02FC08FEA92E060E040E050E00E94E3
:100F1000941080E893E060E042E050E00E9494107A
:100F200014E01FC08FEA92E060E040E050E00E94D1
:100F3000941080E893E060E041E050E00E9494105B
:100F400015E00FC08FEA92E060E040E050E00E94C0
:100F5000941080E893E060E040E050E00E9494103C
:100F600017E010923903D0CD10929E0310927C00AE
:100F700084EC80937A0080917A0084FFFCCF8CEC23
:100F800080937A0008951F920F920FB60F920BB6BE
:100F90000F9211242F934F935F936F937F938F93AF
:100FA0009F93AF93BF93EF93FF93809178009091BD
:100FB0007900AC0160E070E08091430290914402BE
:100FC000A0914502B0914602480F591F6A1F7B1F2E
:100FD000409343025093440260934502709346024B
:100FE000809142028F5F809342028823E1F4209136
:100FF0009E03E22FF0E0EE0FFF1FEA56FC4FBB27E7
:10100000A72F962F852F91838083109243021092F1
:10101000440210924502109246022F5F23702093E3
:101020009E0320937C008CEC80937A00FF91EF91DB
:10103000BF91AF919F918F917F916F915F914F91F0
:101040002F910F900BBE0F900FBE0F901F90189511
:101050009C01F999FECF32BD21BDF89A80B5089563
:1010600085B1817F85B9209A28980000000083B15E
:1010700090E096958795E82FE17083B190E0969582
:10108000879596958795382F317083B190E0F3E07E
:1010900096958795FA95E1F7282F2170289A0000F8
:1010A000000083B143B153B190E09695879581706C
:1010B000E813E2E0842F90E09695879596958795C2
:1010C0008170381332E0852F90E043E09695879544
:1010D0004A95E1F78170281322E083E0389FC00130
:1010E0001124E80F89E0289FC0011124E80FF0E0E7
:1010F000E051FC4FE4918E2F089590E0805790408E
:1011000062E070E00E947C12862F0895FC018381CA
:101110008695869581700895DC0112969C911297B0
:1011200013968C911397890F819514968C9314972D
:1011300020E093E006C0FD01E90FF11D8281280F38
:101140009F5F11968C9111979817A8F3219511968E
:101150008C911197FD01E80FF11D228311968C915E
:1011600011978F5F11968C930895FC0180818E7F7B
:10117000808380818068808385EA8093BC00808141
:1011800080FFFDCF808181FF05C080818D7F8083BE
:1011900081E008958091BC0084FDFCCF85E48093BC
:1011A000BC0080818F77808380E00895DC011296F7
:1011B0008C91129713969C911397980F9195149672
:1011C0008C911497891711F081E0089530E023E0A5
:1011D00005C0EA0FFB1F8281380F2F5FE22FF0E07E
:1011E00011968C91119790E00197E817F9078CF30D
:1011F00031951196EC911197F0E03197EA0FFB1FB2
:101200008281831711F480E0089582E00895CF92DF
:10121000DF92EF92FF920F931F93CF93DF938C0196
:10122000EB01FC01F380F694F694F6E0FF1681F0F2
:10123000FF1528F084E0F81609F0A3C33EC0EAE0E9
:10124000FE1609F4D3C1FCE2FF1609F09AC350C29E
:10125000FC01F780F1E0FF1609F093C38FEA97E0F5
:101260000E94BE0DF80185818A8383818C5F8C7F0B
:101270008B839B8186818370892B8B838091EB028A
:101280008D8386818C7F8E839E8183818370892B61
:101290008E8387818F831886198681E88A87FB86EB
:1012A0001C8681E58D878BE28E878FEF8F87888BF9
:1012B000198A1A8A1B8A82E1FFC2F801878180326B
:1012C00009F463C0813240F48130E1F0813070F084
:1012D000823009F056C33AC0823209F405C1823225
:1012E00008F476C08D3209F04CC321C18FE797E036
:1012F0000E94BE0DF80180858093A00381858093B4
:10130000A10329C08FE497E00E94BE0DF8018581FA
:101310008A8383818C5F8C7F8B839B8186818370A2
:10132000892B8B838091EB028D8386818C7F8E83CA
:101330009E8183818370892B8E8387818F8318861A
:101340008091A00389878091A10340C083E297E048
:101350000E94BE0DF80185818A8383818C5F8C7F1A
:101360008B839B8186818370892B8B838091EB0299
:101370008D8386818C7F8E839E8183818370892B70
:101380008E8387818F831886B1C182EF96E00E9499
:10139000BE0DF80185818A8383818C5F8C7F8B836E
:1013A0009B8186818370892B8B838091EB028D8357
:1013B00086818C7F8E839E8183818370892B8E832F
:1013C00087818F83188688E0898781E08A87ADC00E
:1013D00086EC96E00E94BE0DF80185818A838381A8
:1013E0008C5F8C7F8B839B8186818370892B8B8321
:1013F0008091EB028D8386818C7F8E839E81838199
:101400008370892B8E8387818F8318868285E82E4F
:10141000FF242385922F80E0E82AF92AD484C5840A
:10142000F7E0EF16F10421F48FEF89878A8704C073
:10143000C701019689879A87F701EE0FFF1FEC5EBF
:10144000FD4F0D2D10E060817181600F711FCE0185
:101450000B964C2D50E00E94571285E08D1560F0E0
:10146000C8018C0D911D05973CF0FE01E01BF10BAE
:101470008091EB023E968283EF28C9F4EDE0ED15F2
:1014800078F12D2D30E0C9018C0D911D0D9744F19F
:10149000FE01E21BF30B8091EB0290E0805790403D
:1014A00062E070E00E947C12605A769618C0F9E003
:1014B000FD15B0F02D2D30E0C9018C0D911D09975F
:1014C0007CF0FE01E21BF30B8091EB0290E0805771
:1014D000904062E070E00E947C12605A72966283D3
:1014E00089E0C80EC982E9C186E996E00E94BE0D76
:1014F000F80185818A8383818C5F8C7F8B839B81BC
:1015000086818370892B8B838091EB028D8386810A
:101510008C7F8E839E8183818370892B8E838781CC
:101520008F83188681E089871A8689E0C5C186E69F
:1015300096E00E94BE0DF80185818A8383818C5FCD
:101540008C7F8B839B8186818370892B8B83809199
:10155000EB028D8386818C7F8E839E818381837055
:10156000892B8E8387818F831886108584E00E9463
:101570008404982F1330F9F0143028F41130A9F0B6
:101580001230B0F408C0153001F11530C8F0163033
:1015900009F0D7C11FC0198680EC8A87992311F002
:1015A00081E001C082E08B87CCC180914A021AC0E1
:1015B0008091D60217C080919603909197030EC038
:1015C000809198039091990309C080919A0390911A
:1015D0009B0304C080919C0390919D0396958795F1
:1015E0009695879589871A861B86ABC1FC018781F2
:1015F000813149F1823109F45AC0803109F0C1C109
:1016000086E396E00E94BE0DF80185818A8383817E
:101610008C5F8C7F8B839B8186818370892B8B83EE
:101620008091EB028D8386818C7F8E839E81838166
:101630008370892B8E8387818F8318868CEC8987B2
:101640001A861B8660C18EE096E00E94BE0DF801EE
:1016500085818A8383818C5F8C7F8B839B8186814C
:101660008370892B8B838091EB028D8386818C7FA5
:101670008E839E8183818370892B8E8387818F8364
:101680001886818590E0228513851987722F60E086
:10169000682B792B60507040CE010A96412F50E0A4
:1016A00028E238E00E946012185F198306C185EEB7
:1016B00095E00E94BE0DF80185818A8383818C5F4D
:1016C0008C7F8B839B8186818370892B8B83809118
:1016D000EB028D8386818C7F8E839E8183818370D4
:1016E000892B8E8387818F8380E8888787E0E4C099
:1016F000FC01F780F8E0FF1609F4E1C0FF15B0F037
:1017000085E0F81609F45AC08F1538F0FF2031F142
:10171000E4E0FE1609F031C146C0F6E0FF1609F418
:101720006FC087E0F81609F028C16DC0EAE1FE1627
:1017300009F41DC1EF1548F0FDE0FF1609F403C1DF
:1017400089E1F81609F019C104C1EEE1FE1609F4A9
:10175000FDC0FDE2FF1609F010C10CC18DEB95E054
:101760000E94BE0DF80185818A8383818C5F8C7F06
:101770008B839B8186818370892B8B838091EB0285
:101780008D8386818C7F8E839E8183818370892B5C
:101790008E8387818F831886198684E08A871B86CB
:1017A0001C868BE089C089E995E00E94BE0DF80196
:1017B0008285843009F064C087E0D6C08FE695E06A
:1017C0000E94BE0DF80185818A8383818C5F8C7FA6
:1017D0008B839B8186818370892B8B838091EB0225
:1017E0008D8386818C7F8E839E8183818370892BFC
:1017F0008E8387818F831886198687E08A87F4CE47
:1018000083E495E0BCC089E195E00E94BE0DF8013B
:101810008385482F50E02485922F80E0482B592B58
:101820008285813041F0813018F0823069F406C041
:101830008DE492E005C08FEA92E002C080E893E078
:1018400061E00E9494101CC0F80185818A83838125
:101850008C5F8C7F8B839B8186818370892B8B83AC
:101860008091EB028D8386818C7F8E839E81838124
:101870008370892B8E8387818F838CEC88871AC035
:10188000F80185818A8383818C5F8C7F8B839B8128
:1018900086818370892B8B838091EB028D83868177
:1018A0008C7F8E839E8183818370892B8E83878139
:1018B0008F831886198688E0898381E063C08FEE64
:1018C00094E00E94BE0DF80182858330F0F0F801AB
:1018D00085818A8383818C5F8C7F8B839B818681CA
:1018E0008370892B8B838091EB028D8386818C7F23
:1018F0008E839E8183818370892B8E8387818F83E2
:101900008CEC88871986F982D8CFF80185818A8383
:1019100083818C5F8C7F8B839B8186818370892BF5
:101920008B838091EB028D8386818C7F8E839E8159
:1019300083818370892B8E8387818F831886198694
:101940001A868AE0B9CF82EC94E019C088E994E065
:1019500016C08DE694E00E94BE0DF80185858823AF
:1019600011F081E001C086E08093EA0289CF82E431
:1019700094E005C08AE194E002C08BE094E00E940C
:10198000BE0D80E0DF91CF911F910F91FF90EF90FE
:10199000DF90CF9008951092C5008CE08093C40032
:1019A00088E98093C10010922404109222041092BE
:1019B00023041092A5040895282F80912204909169
:1019C000240481508F779817C1F3E0912404F0E04C
:1019D000EB5DFB4F2083809124048F5F8093240470
:1019E00080912404803811F4109224048091C10065
:1019F00080628093C1000895DC019091230480915E
:101A0000A504981711F481E008959091A504E92F99
:101A1000F0E0EE55FC4F80818C939F5F9093A5047E
:101A20008091A504803811F080E008951092A504FB
:101A300080E008951F920F920FB60F920BB60F928F
:101A400011248F939F93EF93FF93E0912204F0E092
:101A5000EB5DFB4F80818093C600809122048F5FF5
:101A60008093220480912204803811F41092220481
:101A70009091240480912204981729F48091C10048
:101A80008F7D8093C100FF91EF919F918F910F9077
:101A90000BBE0F900FBE0F901F9018951F920F92C4
:101AA0000FB60F920BB60F9211248F939F93EF9363
:101AB000FF9380912304E82FF0E09091C600EE554B
:101AC000FC4F90838F5F80932304809123048038A0
:101AD00011F410922304FF91EF919F918F910F9039
:101AE0000BBE0F900FBE0F901F901895DC013DE0CC
:101AF00040C08A30F1F480912204909124048150F6
:101B00008F779817C1F3E0912404F0E0EB5DFB4F71
:101B10003083809124048F5F809324048091240477
:101B2000803811F4109224048091C1008062809367
:101B3000C1002C91809122049091240481508F77D0
:101B40009817C1F3E0912404F0E0EB5DFB4F208394
:101B5000809124048F5F8093240480912404803832
:101B600011F41092240411968091C1008062809338
:101B7000C1008C91882309F0BCCF0895FC019C0121
:101B80002F5F3F4F44915DE04A30F1F48091220491
:101B90009091240481508F779817C1F3E091240429
:101BA000F0E0EB5DFB4F5083809124048F5F8093C6
:101BB000240480912404803811F41092240480912C
:101BC000C10080628093C10080912204909124041E
:101BD00081508F779817C1F3E0912404F0E0EB5D1A
:101BE000FB4F4083809124048F5F80932404809175
:101BF0002404803811F4109224048091C100806282
:101C00008093C100F9018491882321F02F5F3F4F19
:101C1000482FBACF0895582F40E820E030E070E315
:101C200061E3842F852379F080912204909124042C
:101C300081508F779817C1F3E0912404F0E0EB5DB9
:101C4000FB4F60830EC08091220490912404815048
:101C50008F779817C1F3E0912404F0E0EB5DFB4F20
:101C60007083809124048F5F8093240480912404E6
:101C7000803811F4109224048091C1008062809316
:101C8000C10046952F5F3F4F2830310551F608952A
:101C90000F931F93DF93CF93CDB7DEB728970FB67F
:101CA000F894DEBF0FBECDBFBC01DE011196E4E3A8
:101CB000F2E088E001900D928150E1F7DE0111968B
:101CC00051E08E01075F1F4F2CC04F5F620F731FE3
:101CD00050E068177907C8F75523F9F4809122047A
:101CE0009091240481508F779817C1F3E0912404D8
:101CF000F0E0405DEB5DFB4F4083809124048F5FFB
:101D00008093240480912404803811F410922404D8
:101D10008091C10080628093C1001296A017B10724
:101D200049F08D919C91119740E022273327281B81
:101D3000390BCFCF809122049091240481508F776A
:101D40009817C1F3E0912404F0E0862F805DEB5DED
:101D5000FB4F8083809124048F5F809324048091C3
:101D60002404803811F4109224048091C100806210
:101D70008093C10028960FB6F894DEBF0FBECDBF8A
:101D8000CF91DF911F910F910895DF93CF93CDB73E
:101D9000DEB760970FB6F894DEBF0FBECDBF282F19
:101DA000DE011196E4E2F2E080E101900D928150B3
:101DB000E1F7822F82958F70FE01E80FF11D3181CE
:101DC000809122049091240481508F779817C1F359
:101DD000E0912404F0E0EB5DFB4F3083809124041C
:101DE0008F5F8093240480912404803811F4109232
:101DF00024048091C10080628093C1002F70FE0195
:101E0000E20FF11D218180912204909124048150E0
:101E10008F779817C1F3E0912404F0E0EB5DFB4F5E
:101E20002083809124048F5F809324048091240474
:101E3000803811F4109224048091C1008062809354
:101E4000C10060960FB6F894DEBF0FBECDBFCF9134
:101E5000DF9108951092A9051092A60498E090933E
:101E6000B8008E7F8093BA001092BD0085E4809305
:101E7000BC0008951F920F920FB60F920BB60F92EF
:101E800011248F939F93EF93FF938091B900887FE4
:101E9000883309F470C0893350F4883109F445C09F
:101EA000883209F451C0883009F072C034C08038DB
:101EB000A1F0803A09F1803609F06AC0E0913B0355
:101EC000F0913C0380818068808380818E7F808355
:101ED0008091BB00828381E00CC0E0913B03F091D4
:101EE0003C03809148029091BB00E80FF11D928362
:101EF0008F5F809348020DC0E0913B03F0913C035B
:101F000080914802818380818160808380818F7786
:101F1000808385EC3BC0E091E802F091E9021082F9
:101F200082818093BB0081E00CC0E091E802F091D7
:101F3000E90280914702E80FF11D92819093BB0066
:101F40008F5F8093470221C090914702E091E802A1
:101F5000F091E9028181981729F480818160808362
:101F600085E914C0E90FF11D82818093BB009F5F5A
:101F7000909347020AC0E091E802F091E902808163
:101F80008160808380818260808385E88093BC004B
:101F9000FF91EF919F918F910F900BBE0F900FBE0D
:101FA0000F901F9018958BB18F738BB98AB18F7377
:101FB0008AB90895579A86E0982F9A95F1F7569A1C
:101FC0008A95F1F70895579886E0982F9A95F1F73A
:101FD0005698982F9A95F1F7579A982F9A95F1F766
:101FE000569A8A95F1F70895569886E0982F9A9513
:101FF000F1F757988A95F1F70895582F90E820E067
:1020000030E066E07DE0892F852311F4579A01C006
:10201000579846E0862F8A95F1F75698872F8A952C
:10202000F1F7569A862F8A95F1F796952F5F3F4FD5
:102030002830310541F75798842F8A95F1F7569843
:10204000842F8A95F1F789B1942F9A95F1F7569AD2
:10205000579A942F9A95F1F78095881F8827881FA3
:102060000895579820E030E046E0330F942F9A957A
:10207000F1F75698942F9A95F1F74F993160942F74
:102080009A95F1F7569A942F9A95F1F72F5F283089
:1020900061F7882311F0579A01C0579886E0982F6E
:1020A0009A95F1F756989DE09A95F1F7569A579AB6
:1020B0008A95F1F7832F0895EF92FF920F931F9364
:1020C000CF93DF93182FEB010E94DA0F812F8160ED
:1020D0000E94FD0F882321F40E94F40F81E011C0BB
:1020E00081E00E943110182F00E080E00E94311042
:1020F000E82E0E94F40FFF240E291F29198308835C
:1021000080E0DF91CF911F910F91FF90EF900895A4
:10211000FC011086128671836083128213825583BC
:102120004483168217820895DC016623C9F412964F
:102130008C91129790E0880F991FED91FC91119767
:10214000E80FF91F5183408312968C9112978F5F8D
:1021500012968C9312978430E1F412961C92089593
:1021600016968C91169790E0880F991F1496ED9112
:10217000FC911597E80FF91F5183408316968C91B7
:1021800016978F5F16968C931697843011F41696D7
:102190001C920895CF93DF93DC01EA01662309F5D1
:1021A00013969C91139712968C9112979817D9F1C8
:1021B000892F90E0880F991FED91FC911197E80FFE
:1021C000F91F808191819983888313968C9113974D
:1021D0008F5F13968C931397843039F513961C9266
:1021E00024C017969C91179716968C91169798175E
:1021F000D1F0892F90E0880F991F1496ED91FC91F2
:102200001597E80FF91F808191819983888317962C
:102210008C9117978F5F17968C931797843029F4BA
:1022200017961C9202C081E001C080E0DF91CF913F
:102230000895DF92EF92FF920F931F93DF93CF9356
:1022400000D0CDB7DEB78C01FC018085882309F072
:10225000B8C02285213041F0213070F0223091F059
:10226000233009F048C027C095B1F80181858095D9
:10227000892385B927873FC085B1F8019185892BCE
:1022800085B937C0F8012585222341F095B18185B4
:102290008095892385B9215025870AC0F8012685B4
:1022A000222331F085B19185892B85B9215026876C
:1022B000F801868518C0F8012685222339F085B1FA
:1022C0009185892B85B9215026870BC0F80125857A
:1022D000222339F095B181858095892385B92150D4
:1022E0002587F8018585882331F483858587848552
:1022F000868781E08787F801D784F1E0DF1609F04F
:10230000CCC0C80161E07E010894E11CF11CA7016A
:102310000E94CA10882321F5F801D08649815A818C
:102320009A0130702115310511F4108A47C0C90196
:1023300001978A3F910540F482E0F801808B518B30
:10234000428B538B448B3AC02C3F310519F4F80172
:10235000108634C02F3F310589F5F801D08A2EC090
:10236000C80160E0A7010E94CA10882339F589815D
:102370009A8190708130910549F08130910548F043
:102380008230910549F00397C9F40FC0F801D28655
:1023900015C0F801128612C09AE0F80193878AE509
:1023A00084879587868782E008C09AE5F80193873D
:1023B0008AE084879587868783E08287F80117867D
:1023C0006CC0F8012089213039F0213068F02230CA
:1023D00089F0233079F519C095B1F8018185809590
:1023E000892385B9258B26C085B1F8019185892B74
:1023F00085B91EC0F8012489222339F085B1918561
:10240000892B85B92150248B0BC0F8012389222305
:1024100039F095B181858095892385B92150238B29
:10242000F8018389882331F48189838B8289848BA5
:1024300081E0858BF8018589882379F1C80161E005
:10244000AE014F5F5F4F0E94CA10882321F561E003
:10245000F801608749815A819A0130702115310550
:1024600011F4108A18C0C90101978A3F910540F400
:1024700082E0F801808B518B428B538B448B0BC0D5
:102480002C3F310519F4F801108605C02F3F3105A6
:1024900011F4F801608BF801158A0F900F90CF911D
:1024A000DF911F910F91FF90EF90DF900895FB0156
:1024B000DC0102C005900D9241505040D8F70895BC
:1024C000A0E0B0E0E6E6F2E10C94AD127C01EB0195
:1024D0008A01690109C0CE012196F6010995F7012B
:1024E00081937F010150104001151105A1F7CDB76F
:1024F000DEB7E8E00C94C91297FB092E07260AD034
:1025000077FD04D00CD006D000201AF470956195A8
:102510007F4F0895F6F7909581959F4F0895AA1BD8
:10252000BB1B51E107C0AA1FBB1FA617B70710F0BE
:10253000A61BB70B881F991F5A95A9F780959095F0
:10254000BC01CD0108952F923F924F925F926F92FE
:102550007F928F929F92AF92BF92CF92DF92EF9233
:10256000FF920F931F93CF93DF93CDB7DEB7CA1BB4
:10257000DB0B0FB6F894DEBF0FBECDBF09942A88DF
:10258000398848885F846E847D848C849B84AA8487
:10259000B984C884DF80EE80FD800C811B81AA8114
:1025A000B981CE0FD11D0FB6F894DEBF0FBECDBFDF
:0825B000ED010895F894FFCF3E
:1025B8004D6F64756C6520416464726573733A206D
:1025C800000A0A00190230027002B002F002300359
:1025D8007003B0033031323334353637383941423D
:0C25E800434445461027E80364000A0045
:00000001FF
